 libOpenVGU

 Timestamp is 4be8c529 (Tue May 11 11:47:05 2010)

 Preferred load address is 10000000

 Start         Length     Name                   Class
 0001:00000000 00000004H .CRT$XCA                CODE
 0001:00000004 00000004H .CRT$XCZ                CODE
 0001:00000008 00000004H .CRT$XIA                CODE
 0001:0000000c 00000004H .CRT$XIZ                CODE
 0001:00000010 00000004H .CRT$XPA                CODE
 0001:00000014 00000004H .CRT$XPZ                CODE
 0001:00000018 00000004H .CRT$XTA                CODE
 0001:0000001c 00000004H .CRT$XTZ                CODE
 0001:00000020 0000001cH .rdata                  CODE
 0001:0000003c 00000027H .rdata$debug            CODE
 0001:00000064 00002b64H .text                   CODE
 0001:00002bc8 0000001cH .xdata                  CODE
 0001:00002be4 00000028H .idata$2                CODE
 0001:00002c0c 00000014H .idata$3                CODE
 0001:00002c20 0000008cH .idata$4                CODE
 0001:00002cac 00000060H .idata$6                CODE
 0001:00002d10 00000119H .edata                  CODE
 0002:00000000 0000008cH .idata$5                DATA
 0002:0000008c 00000008H .data                   DATA
 0002:00000094 00000010H .bss                    DATA
 0003:00000000 000000c8H .pdata                  DATA

  Address         Publics by Value              Rva+Base       Lib:Object

 0000:00000000       ___safe_se_handler_count   00000000     <absolute>
 0000:00000000       ___safe_se_handler_table   00000000     <absolute>
 0001:00000000       __xc_a                     10001000     corelib0:crt0init.obj
 0001:00000004       __xc_z                     10001004     corelib0:crt0init.obj
 0001:00000008       __xi_a                     10001008     corelib0:crt0init.obj
 0001:0000000c       __xi_z                     1000100c     corelib0:crt0init.obj
 0001:00000010       __xp_a                     10001010     corelib0:crt0init.obj
 0001:00000014       __xp_z                     10001014     corelib0:crt0init.obj
 0001:00000018       __xt_a                     10001018     corelib0:crt0init.obj
 0001:0000001c       __xt_z                     1000101c     corelib0:crt0init.obj
 0001:000003d4       vguLine                    100013d4 f   vgu.obj
 0001:00000464       vguPolygon                 10001464 f   vgu.obj
 0001:000005c0       vguRect                    100015c0 f   vgu.obj
 0001:00000714       vguRoundRect               10001714 f   vgu.obj
 0001:000009b8       vguEllipse                 100019b8 f   vgu.obj
 0001:00000b44       vguArc                     10001b44 f   vgu.obj
 0001:00001e8c       vguComputeWarpSquareToQuad 10002e8c f   vgu.obj
 0001:00002500       vguComputeWarpQuadToSquare 10003500 f   vgu.obj
 0001:000025e0       vguComputeWarpQuadToQuad   100035e0 f   vgu.obj
 0001:0000275c       vgGetError                 1000375c f   libOpenVG:libOpenVG.dll
 0001:0000276c       vgGetParameteri            1000376c f   libOpenVG:libOpenVG.dll
 0001:0000277c       vgGetParameterf            1000377c f   libOpenVG:libOpenVG.dll
 0001:0000278c       vgAppendPathData           1000378c f   libOpenVG:libOpenVG.dll
 0001:0000279c       DllMain                    1000379c f   corelib0:dllmain.obj
 0001:000028b8       _DllMainCRTStartup         100038b8 f   corelib0:pegdmain.obj
 0001:000028e8       __GSHandlerCheckCommon     100038e8 f   corelib0:gshandler.obj
 0001:00002924       __GSHandlerCheck           10003924 f   corelib0:gshandler.obj
 0001:00002948       __security_init_cookie     10003948 f   corelib0:seccinit.obj
 0001:000029a4       __security_check_cookie    100039a4 f   corelib0:armsecgs.obj
 0001:000029b8       __gsfailure                100039b8 f   corelib0:armsecgs.obj
 0001:00002ac4       _cexit                     10003ac4 f   corelib0:cexit.obj
 0001:00002ae0       _initterm                  10003ae0 f   corelib0:crt0dat.obj
 0001:00002b14       _cinit                     10003b14 f   corelib0:crt0dat.obj
 0001:00002b48       malloc                     10003b48 f   corelib1:COREDLL.dll
 0001:00002b58       free                       10003b58 f   corelib1:COREDLL.dll
 0001:00002b68       _XcptFilter                10003b68 f   corelib1:COREDLL.dll
 0001:00002b78       __C_specific_handler       10003b78 f   corelib1:COREDLL.dll
 0001:00002b88       __security_gen_cookie2     10003b88 f   corelib1:COREDLL.dll
 0001:00002b98       __report_gsfailure         10003b98 f   corelib1:COREDLL.dll
 0001:00002ba8       DisableThreadLibraryCalls  10003ba8 f   coredll:COREDLL.dll
 0001:00002bb8       TerminateProcess           10003bb8 f   coredll:COREDLL.dll
 0001:00002be4       __IMPORT_DESCRIPTOR_libOpenVG 10003be4     libOpenVG:libOpenVG.dll
 0001:00002bf8       __IMPORT_DESCRIPTOR_COREDLL 10003bf8     corelib1:COREDLL.dll
 0001:00002c0c       __NULL_IMPORT_DESCRIPTOR   10003c0c     libOpenVG:libOpenVG.dll
 0002:00000000       __imp_cos                  10004000     corelib1:COREDLL.dll
 0002:00000004       __imp_DisableThreadLibraryCalls 10004004     coredll:COREDLL.dll
 0002:00000008       __imp_malloc               10004008     corelib1:COREDLL.dll
 0002:0000000c       __imp___subs               1000400c     corelib1:COREDLL.dll
 0002:00000010       __imp___divs               10004010     corelib1:COREDLL.dll
 0002:00000014       __imp___adds               10004014     corelib1:COREDLL.dll
 0002:00000018       __imp___stod               10004018     corelib1:COREDLL.dll
 0002:0000001c       __imp_floor                1000401c     corelib1:COREDLL.dll
 0002:00000020       __imp___dtoi               10004020     corelib1:COREDLL.dll
 0002:00000024       __imp_free                 10004024     corelib1:COREDLL.dll
 0002:00000028       __imp___les                10004028     corelib1:COREDLL.dll
 0002:0000002c       __imp___negs               1000402c     corelib1:COREDLL.dll
 0002:00000030       __imp___muls               10004030     corelib1:COREDLL.dll
 0002:00000034       __imp___lts                10004034     corelib1:COREDLL.dll
 0002:00000038       __imp___gts                10004038     corelib1:COREDLL.dll
 0002:0000003c       __imp_TerminateProcess     1000403c     coredll:COREDLL.dll
 0002:00000040       __imp_sin                  10004040     corelib1:COREDLL.dll
 0002:00000044       __imp___dtos               10004044     corelib1:COREDLL.dll
 0002:00000048       __imp___eqs                10004048     corelib1:COREDLL.dll
 0002:0000004c       __imp___eqd                1000404c     corelib1:COREDLL.dll
 0002:00000050       __imp___ltd                10004050     corelib1:COREDLL.dll
 0002:00000054       __imp___gtd                10004054     corelib1:COREDLL.dll
 0002:00000058       __imp___muld               10004058     corelib1:COREDLL.dll
 0002:0000005c       __imp___subd               1000405c     corelib1:COREDLL.dll
 0002:00000060       __imp___divd               10004060     corelib1:COREDLL.dll
 0002:00000064       __imp__XcptFilter          10004064     corelib1:COREDLL.dll
 0002:00000068       __imp___C_specific_handler 10004068     corelib1:COREDLL.dll
 0002:0000006c       __imp___security_gen_cookie2 1000406c     corelib1:COREDLL.dll
 0002:00000070       __imp___report_gsfailure   10004070     corelib1:COREDLL.dll
 0002:00000074       \177COREDLL_NULL_THUNK_DATA 10004074     corelib1:COREDLL.dll
 0002:00000078       __imp_vgAppendPathData     10004078     libOpenVG:libOpenVG.dll
 0002:0000007c       __imp_vgGetParameterf      1000407c     libOpenVG:libOpenVG.dll
 0002:00000080       __imp_vgGetParameteri      10004080     libOpenVG:libOpenVG.dll
 0002:00000084       __imp_vgGetError           10004084     libOpenVG:libOpenVG.dll
 0002:00000088       \177libOpenVG_NULL_THUNK_DATA 10004088     libOpenVG:libOpenVG.dll
 0002:0000008c       __security_cookie          1000408c     corelib0:seccinit.obj
 0002:00000090       __security_cookie_complement 10004090     corelib0:seccinit.obj
 0002:00000094       _exitflag                  10004094     corelib0:cexit.obj
 0002:00000098       __onexitend                10004098     <common>
 0002:0000009c       __onexitbegin              1000409c     <common>
 0002:000000a0       _pRawDllMain               100040a0     <common>

 entry point at        0001:000028b8

 Static symbols

 0001:00000064       OVGNormaliseData           10001064 f   vgu.obj
 0001:00000370       OVG_VGU_Error              10001370 f   vgu.obj
 0001:000014cc       OVG_VGU_mx3d_mul           100024cc f   vgu.obj
 0001:0000198c       OVG_VGU_mx3d_invert        1000298c f   vgu.obj
 0001:000027bc       _DllMainCRTStartupHelper   100037bc f   corelib0:pegdmain.obj
 0001:000029fc       doexit                     100039fc f   corelib0:cexit.obj
